:04000000CCEF13F03E
:1000080000C016F001C015F0E1CF17F0E2CF18F0EC
:100018009EAA61D09DAA5FD00FEC0DF000C040F100
:10002800ABA20ED0AB98010E01013325006E000E75
:100038003421016E00C033F101C034F1AB88406B4C
:10004800ABA411D00101AB9E010E3325006E000E4A
:100058003421016E00C033F101C034F1AB8E0FECD6
:100068000DF000C040F1010140510D0A09E0000EF9
:10007800006E4551005C02E144517F0801E313D052
:10008800010E2C6E000E2D6EA10E4425E16E000EA1
:100098004521E26EE66A9D9A44C13DF145C13EF1B3
:1000A800446B456B18D02C6A2D6AA10E4425E16E6D
:1000B800000E4521E26E40C1E6FF44C13DF145C155
:1000C8003EF1010E4425006E000E4521016E00C070
:1000D80044F101C045F1F2AA09D0F2A407D0D59E97
:1000E800F29AF294010E306E000E316E16C000F0D6
:0E00F80015C001F017C0E1FF18C0E2FF1100B3
:080106000AAE029E000E120079
:10010E000B840BAE92EF00F0010E036E026A016AD1
:0A011E00006A0A360232FF0E1200DA
:0E012800026A016A006A086A036A000E120089
:100136000B820BAEA5EF00F0036802680168006849
:080146000A360232FF0E12001E
:10014E000CB0E9EF00F00CA28FEF01F00E6A000E7A
:10015E00026400EF01F0F00E0214D8A4CBEF00F011
:10016E00023A01380F0B02260138F00B016E0038EF
:10017E000F0B01260038F00B006E08380F0B00260F
:10018E000838F00B086E0E84D89002BEE4EF00F033
:10019E0008360036013602360E2A02BEE4EF00F0B3
:1001AE0008360036013602360E2A02BEE4EF00F0A3
:1001BE0008360036013602360E2A0E50036485EFDD
:1001CE0001F0035E0BBC08AE8AEF01F0D880800E02
:1001DE0008640030000E002201220222D8A08AEF0D
:1001EE0001F0023201320032034A8FEF01F08AEF42
:1001FE0001F001C002F000C001F008C000F0086A72
:10020E00000E0E86026437EF01F0F00E0214D8A431
:10021E001FEF01F0023A01380F0B02260138F00BE6
:10022E00016E00380F0B01260038F00B006E0E84A5
:10023E00D89002BEE4EF00F00036013602360E2AE8
:10024E0002BEE4EF00F00036013602360E2A02BE80
:10025E00E4EF00F00036013602360E2AE4EF00F02D
:10026E0001C002F000C001F0006A000E0E960E886A
:10027E00026464EF01F0F00E0214D8A44FEF01F007
:10028E00023A01380F0B02260138F00B016E0E8474
:10029E00D89002BEE4EF00F0013602360E2A02BEFE
:1002AE00E4EF00F0013602360E2A02BEE4EF00F053
:1002BE00013602360E2AE4EF00F001C002F0016AA8
:1002CE00000E0E86026494EF01F0F00E0214D8A414
:1002DE0073EF01F0023A0E84D89002BEE4EF00F004
:1002EE0002360E2A02BEE4EF00F002360E2A02BEDD
:1002FE00E4EF00F002360E2AE4EF00F0010E0C6E71
:10030E00FFDE97EF01F0020E0C6EF6DE97EF01F0B6
:10031E00040E0C6E09DF97EF01F0080E0C6EFDDE79
:02032E001200BB
:10033000025006180E6E086A096A0B6A03500764B9
:100340008BEF02F006500A6E068E028E03500B6E83
:100350000750036E000E0B64DBEF01F00B50075EDD
:10036000D8B47CEF02F0070E07644AEF02F0075E94
:1003700000C008F001C000F002C001F0026A074EA0
:100380007CEF02F007641FEF02F0075E00C008F088
:1003900001C000F0016A074E7CEF02F00764FDEF38
:1003A00001F0075E00C008F0006A074E7CEF02F023
:1003B0000764E4EF01F00AC002F005C001F004C0D8
:1003C00000F0086AA5EF03F0030E0764EFEF01F0F9
:1003D000075E08380F0B086E074E7CEF02F0D890CE
:1003E0000832074E7CEF02F0D8900832074E7CEFBF
:1003F00002F0D89008327CEF02F0030E07640EEF93
:1004000002F0075E08380F0B086E0038F00B082664
:1004100000380F0B006E074E7CEF02F0D8900032D0
:100420000832074E7CEF02F0D89000320832074EB7
:100430007CEF02F0D890003208327CEF02F0030E1D
:10044000076436EF02F0075E08380F0B086E0038BD
:10045000F00B082600380F0B006E0138F00B002659
:1004600001380F0B016E074E7CEF02F0D89001327D
:1004700000320832074E7CEF02F0D8900132003291
:100480000832074E7CEF02F0D89001320032083279
:100490007CEF02F0030E076467EF02F0075E083896
:1004A0000F0B086E0038F00B082600380F0B006E9B
:1004B0000138F00B002601380F0B016E0238F00BEB
:1004C000012602380F0B026E074E7CEF02F0D89027
:1004D0000232013200320832074E7CEF02F0D8902F
:1004E0000232013200320832074E7CEF02F0D8901F
:1004F0000232013200320832096A000E0EAE70EF8D
:1005000003F0081E001E011E021E082A00220122FE
:10051000022270EF03F00750D8A491EF02F0A5EF8C
:1005200003F0096A02C00AF0028E068E0750035CCF
:10053000076ED8B463EF03F0070E076431EF03F0E2
:10054000075E0450096E0550046E0650056E066A7B
:10055000074E63EF03F0070E076406EF03F0075E34
:100560000450096E0550046E056A074E63EF03F0F0
:10057000070E0764E4EF02F0075E0450096E046A98
:10058000074E63EF03F0070E0764CBEF02F00AC0DB
:1005900002F0A5EF03F0030E0764D6EF02F0075E4A
:1005A00009380F0B096E074E63EF03F0D89009323C
:1005B000074E63EF03F0D8900932074E63EF03F064
:1005C000D890093263EF03F0030E0764F5EF02F0F1
:1005D000075E09380F0B096E0438F00B0926043842
:1005E0000F0B046E074E63EF03F0D890043209320C
:1005F000074E63EF03F0D89004320932074E63EFE1
:1006000003F0D8900432093263EF03F0030E07645D
:100610001DEF03F0075E09380F0B096E0438F00B6D
:10062000092604380F0B046E0538F00B0426053834
:100630000F0B056E074E63EF03F0D89005320432BE
:100640000932074E63EF03F0D890053204320932C5
:10065000074E63EF03F0D89005320432093263EF9E
:1006600003F0030E07644EEF03F0075E09380F0B2B
:10067000096E0438F00B092604380F0B046E053898
:10068000F00B042605380F0B056E0638F00B052617
:1006900006380F0B066E074E63EF03F0D890063254
:1006A000053204320932074E63EF03F0D890063268
:1006B000053204320932074E63EF03F0D890063258
:1006C000053204320932086A000E0EAE70EF03F0F4
:1006D000091E041E051E061E092A042205220622E2
:1006E000095008260450002205500122065002221B
:1006F0000EBE87EF03F0D8A096EF03F0023201326E
:1007000000320832033E96EF03F0A0EF03F0D8B0BA
:100710009BEF03F0000E081E001E011E021E082A99
:100720000022012202220A7E9BEF03F0010E0C6ED2
:100730000EDDA7EF03F0020E0C6E09DDA7EF03F04C
:10074000040E0C6EF8DCA7EF03F0000E0C6E120026
:100750000B800BAEB4EF03F0026A0AAEFF0E026E1E
:0C076000016E006E0A360232FF0E12001D
:08076C000B6A0B86FF0E120060
:100774000B6A0A6A096A00500402F4CF09F0F3CF45
:1007840008F001500502F4CF0BF0F3CF0AF000504B
:100794000502F3500926F4500A22E86A0B2201509C
:1007A4000402F3500926F4500A22E86A0B2208C016
:1007B40000F009C001F00AC002F00BC003F01200FF
:1007C400026A036A800E0318006E800E005C02E168
:1007D400080E025C21E28B96020E0D6E0D2EFED7E2
:1007E4000000800E04018015016E0150800A02E1B0
:1007F4008B8801D08B98020E0D6E04010D2EFDD74F
:1008040000008B8680378091020E0D6E0D2EFED770
:0A0814000000024A032AD6D71200A2
:10081E0000C008F00B6A0C6A9E0E036E0A6A026A2A
:0C082E00016A006A020E0C6E8BDC1200E6
:10083A000450000A12E10550000A0FE10650000AAE
:10084A000CE10750000A09E1FF0E006EFF0E016E6F
:10085A007F0E026EFF0E036EA7D0086A096A075060
:10086A00D8B4C8EF04F00350D8B4CCEF04F0025067
:10087A0006180A6E028E068E0E6A02C008F001C0C1
:10088A000CF000C00DF004500D5E0550D8A0053CD8
:10089A000C5E0650D8A0063C085E086A0C6A0D6A0F
:1008AA00D8A05FEF04F0D890023201320032083249
:1008BA00010E0E6E0750035ED8A06CEF04F07E0E98
:1008CA000E240326D8B0D1EF04F072EF04F07E0EA6
:1008DA000E240326D8A0D6EF04F0180E0B6E0D36A0
:1008EA000C3608360036013602360E360450005EE3
:1008FA000550D8A0053C015E0650D8A0063C025E11
:10090A0006340E120EA08DEF04F00D8098EF04F05D
:10091A00045000260550D8B0053C01260650D8B030
:10092A00062802260D900B2E74EF04F0BEEF04F099
:10093A00D8900036013602360E360450005E055055
:10094A00D8A0053C015E0650D8A0063C025E0634DB
:10095A000E10010B0D26D8B00C2AD8B4082AD8A438
:10096A00BEEF04F008320C320D32032AD8B4D1EFAC
:10097A0004F00AAE089E0850026E0C50016E0D502B
:10098A00006ED9EF04F0010EECDED9EF04F0020E8E
:10099A0094EC00F0D9EF04F0040E9BEC00F0D9EFD0
:0A09AA0004F0080E87EC00F01200C4
:1009B4008B82020E0D6E0D2EFED700008B90020E60
:1009C4000D6E0D2EFED700007BC480F4F9DE8B8003
:0209D40012000F
:1009D6000C6A0E6A0250D8A404EF05F001C002F0BA
:1009E60000C001F0006A0E860250D8A404EF05F09C
:1009F60001C002F0016A0E960E880250D8B416EFB6
:100A060005F00E50035ED8A4D8A01CEF05F0D890D0
:100A160002BE22EF05F0003601360236032E0BEF3A
:100A260005F01CEF05F0010E0C6E94EC00F026EFBD
:100A360005F0020E0C6E87EC00F026EF05F0040EB2
:080A46000C6E83EC00F01200BD
:100A4E008B928B907BC480F4B6DE060E0C6E300E4D
:100A5E000D6E0D2EFED70C2EFCD700008B801200D3
:100A6E00086A096A000E07620364BCEF05F00250C3
:100A7E0006180A6E075003267E0ED8A04DEF05F01D
:100A8E00035ED8B0C1EF05F051EF05F0035ED8A0BC
:100A9E00C6EF05F0028E068E02C00EF001C00BF0FE
:100AAE0000C00DF000500402F4CF0CF0015005020E
:100ABE00F4CF00F0F3CF08F00402F3500C26F450FC
:100ACE000822000E00220D500502F3500C26F450A1
:100ADE000822000E002202500402F3500826F450A1
:100AEE00002202500502016A000E0122F350002678
:100AFE00F45001220D500602F3500826F450002245
:100B0E00026A000E012202220B500602F35000264A
:100B1E00F4500122000E02220E500602F35001265E
:100B2E00F450022202BEA4EF05F00836003601365C
:100B3E0002360306D8B4C6EF05F0B7EF05F0D8803D
:100B4E00800E08640030000E002201220222D8A07E
:100B5E00B7EF05F0023201320032034AC1EF05F061
:100B6E000AAE029E000EC9EF05F0010E94EC00F0E5
:100B7E00C9EF05F0020E9BEC00F0C9EF05F0040E74
:060B8E0087EC00F01200EC
:100B94000B6A0C6A0A6A0350D8B4FFEF05F00A9E88
:100BA400028E860E035E03BEDDEF05F0D8B4DDEFE2
:100BB40005F002EF06F0036C080E035CD8A0EBEF1F
:100BC40005F0036E0236026A0350D8A4D890F4EFFD
:100BD40005F00350D8B4F4EF05F0D8900232032E98
:100BE400EFEF05F00BBC02A0FFEF05F0D8A0FFEF7C
:100BF40005F0022AD8B409EF06F0016A0EEF06F0F8
:100C04000B800BAE12EF06F0016A12EF06F0010E34
:100C14000C6E9CDD14EF06F0000E0C6E14EF06F063
:0A0C2400FF0E0C6E0250006E12006D
:080C2E00067E98EC01F01200B3
:100C36000050086E0150006E0250016E0350026EA5
:100C4600036A0B6A0C6A9E0E036E0A6A02AE38EFDE
:100C560006F0081E001E011E021E082AD8B4002A2D
:100C6600D8B4012AD8B4022A0A8E020E0C6EA7EC5A
:040C760000F0120078
:100C7A000A6A0350D8A40A800750D8A40A820A50E4
:100C8A00D8B4A0EF06F0030AD8B459EF06F00AB0B8
:100C9A0054EF06F006AE9EEF06F09CEF06F002AEA9
:100CAA009CEF06F09EEF06F00250800B0A6E029E41
:100CBA000650800B069E0A18D8B46AEF06F00A504E
:100CCA00D8B49CEF06F09EEF06F00750035CD8B448
:100CDA0074EF06F0D8A090EF06F096EF06F00650F3
:100CEA00025CD8B47EEF06F0D8A090EF06F096EF3B
:100CFA0006F00550015CD8B488EF06F0D8A090EF52
:100D0A0006F096EF06F00450005CD8B4A0EF06F0A7
:100D1A00D8B096EF06F00A52D8B49EEF06F09CEFD0
:100D2A0006F00A52D8B49CEF06F09EEF06F0D8807F
:0E0D3A001200D8901200D880D8841200120047
:100D48007CC400F00032009E0032009E0032009EFB
:100D5800000E016E600E046E000E056E07DD0401C4
:100D68007B5100247E6F000E01207F6F7D5320E0B1
:100D7800480E7E25026E010E7F21036E070E7C153C
:100D8800006E00C001F0010E006E015004E0003654
:100D98000090FF0FFBD702C0E9FF03C0EAFFEE5047
:100DA800001202C0E1FF03C0E2FF00C0E6FF22D04C
:100DB800480E7E25026E010E7F21036E070E7C15FC
:100DC800006E00C001F0010E006E015004E0003614
:100DD8000090FF0FFBD70050FF08006E02C0E9FF2C
:100DE80003C0EAFFEE50001602C0E1FF03C0E2FFB5
:060DF80000C0E6FF12003E
:100DFE000B6A0C6A086A0350D8B483EF07F002C07E
:100E0E000AF0028E9E0E035E03AE73EF07F0036CC4
:100E1E00080E035CD8A040EF07F0036E083600C042
:100E2E0008F001C000F002C001F0026A080E035C77
:100E3E00D8A040EF07F0036E083600C008F001C0DE
:100E4E0000F0016A080E035CD8A040EF07F0036EB5
:100E5E00083600C008F0006A080E035CD8A040EF08
:100E6E0007F0036E0836086A0350D8A4D8904CEFEA
:100E7E0007F00350D8B44CEF07F0D890023201328D
:100E8E0000320832032E44EF07F00BBC08A05DEFD2
:100E9E0007F0D8A05DEF07F0082AD8B4002AD8B41E
:100EAE00012AD8B4022A02BE87EF07F00AAE83EFFA
:100EBE0007F0021E011E001E081E082AD8B4002AC2
:100ECE00D8B4012AD8B4022A83EF07F0026A016A65
:100EDE00006A086A83EF07F00B800BAE8DEF07F008
:100EEE00026A0AAE8DEF07F0026E016E006E086E9A
:100EFE000A3602328DEF07F00C6A000E8EEF07F005
:100F0E00010E0C6E000E1DDC8EEF07F0FF0E025070
:100F1E00036E0150026E0050016E0850006E1200FA
:0E0F2E00ACB202D00000FCD75BC4ADFF1200D5
:100F3C0004015B51390806E3300E5B5D03E3010EDF
:080F4C00006E01D0006A1200E2
:100F540062C400F063C401F0000E040163BFFF0E1D
:100F6400026E036E003600900136023603360036F8
:100F740000900136023603365F510024F66E60514C
:100F84000120F76E61510220F86E0900F5CF64F478
:100F94000900F5CF65F40900F5CF66F40900F5CF33
:100FA40067F46251631148E05BC400F05CC401F073
:100FB4005DC402F05EC403F064C404F065C405F0CB
:100FC40066C406F067C407F050DD010E625F000ED0
:100FD400635B62C404F063C405F0000E63BFFF0EDC
:100FE400066E076E04360490053606360736043658
:100FF40004900536063607365F510424F66E6051B8
:101004000520F76E61510620F86E0900F5CF04F053
:101014000900F5CF05F00900F5CF06F00900F5CF7A
:1010240007F098EC01F000C064F401C065F402C05C
:1010340066F403C067F4B5D764C400F065C401F076
:0A10440066C402F067C403F0120056
:10104E00A69C5CC4AAFF5BC4A9FFA69EA680A8CFDF
:04105E0000F012008C
:10106200400E04017B6FF2DC800E04017B6FEEDC2C
:10107200340E0C6EF10E0D6E0D2EFED70C2EFCD71B
:101082000000000004015B6B5C6B800E5C19006E5B
:10109200800E030A005C02E1000E5B5D0FE27B6BD7
:1010A20088DC060E0C6E300E0D6E0D2EFED70C2E49
:1010B200FCD7000004015B4B5C2BE7D7400E7B6F33
:0C10C200C5DC800E04017B6FC1DC120055
:1010CE005EC400F0016A026A036AFF0E0016000E8B
:1010DE00011600C063F401C064F47F0E005C026E62
:1010EE00000E0158036E02C063F403C064F4800E58
:1010FE000318006E800E005C02E1000E025C21E21D
:10110E00046A056A066A076A5BC400F05CC401F0F3
:10111E005DC402F05EC403F0A9DD010ED8B0000E6E
:10112E00006E005209E0000E006E000E016E800E81
:10113E00026E7F0E036E5AD0006A016A026A036A5B
:10114E0055D0000E006E04016451005C02E1635143
:10115E00180809E25BC400F05CC401F05DC402F043
:10116E005EC403F043D05BC400F05CC401F05DC408
:10117E0002F05EC403F03CDE57DD00C05FF401C038
:10118E0060F402C061F403C062F400C004F001C058
:10119E0005F002C006F003C007F05BC400F05CC4AB
:1011AE0001F05DC402F05EC403F060DD010ED8B044
:1011BE00000E006E005212E0000E046E000E056E60
:1011CE00000E066E7F0E076E5FC400F060C401F065
:1011DE0061C402F062C403F023DD08D05FC400F0E6
:0E11EE0060C401F061C402F062C403F012009C
:0A11FC001D0E0D6E0D2EFED7120021
:101206000B6A0C6A0A6A0350D8B44DEF09F0028ED5
:101216008E0E035E03BE15EF09F0D8B415EF09F084
:1012260051EF09F0036C080E035CD8A02CEF09F00F
:10123600036E013602C001F0026A080E035CD8A0F4
:101246002CEF09F00136016A0350D8A4D89036EF86
:1012560009F00350D8B436EF09F0D89002320132C3
:10126600032E30EF09F00BBC01A043EF09F0D8A024
:1012760043EF09F0012AD8B4022A02BE60EF09F052
:101286000AAE66EF09F0021E011E012AD8B4022A30
:1012960066EF09F0026A016A66EF09F00B800BAE91
:1012A6006AEF09F0026A0AAE6AEF09F0FF0E026EF3
:1012B600016E0A3602326AEF09F0010E0C6EA8ECD6
:1012C60003F06CEF09F0000E0C6E6CEF09F0FF0EE8
:0C12D6000C6E0150006E0250016E120000
:1012E2000050086E0150006E016A026A036A0B6ABE
:1012F2000C6A960E036E0A6A00C001F008C000F084
:0A130200086A026AEBEC04F0120026
:10130C0004016A6B6B6B6C6B6D6B6E6B6F6B706BE4
:10131C00716B5C515E5D0DE25EC464F45CC466F49A
:10132C00000E6E6F000E6F6F800E706F7F0E716F00
:10133C000CD05CC464F45EC466F4000E6E6F000ED8
:10134C006F6F000E706F7F0E716F5C515E1904E150
:10135C006E6B6F6B706B716B5B515D5D0DE25DC4A1
:10136C0063F45BC465F4000E6A6F000E6B6F800E45
:10137C006C6F7F0E6D6F0CD05BC463F45DC465F451
:10138C00000E6A6F000E6B6F000E6C6F7F0E6D6F30
:10139C005B515D1904E16A6B6B6B6C6B6D6B63512C
:1013AC00655D006E0050010F026E02C061F4645165
:1013BC00665D006E0050010F016E01C062F40250B8
:1013CC00015C37E262C400F00FEC04F000C072F470
:1013DC0001C073F402C074F403C075F461C400F06E
:1013EC000FEC04F000C004F001C005F002C006F0E0
:1013FC0003C007F072C400F073C401F074C402F0AF
:10140C0075C403F01DEC04F06EC404F06FC405F059
:10141C0070C406F071C407F037EC05F000C06EF430
:10142C0001C06FF402C070F403C071F461C467F4BE
:10143C0036D061C400F00FEC04F000C072F401C0AF
:10144C0073F402C074F403C075F462C400F00FECC2
:10145C0004F000C004F001C005F002C006F003C0A7
:10146C0007F072C400F073C401F074C402F075C4C8
:10147C0003F01DEC04F06AC404F06BC405F06CC4FA
:10148C0006F06DC407F037EC05F000C06AF401C03B
:10149C006BF402C06CF403C06DF462C467F4040115
:1014AC00606B6751605DD8B07CD060C400F00FEC0D
:1014BC0004F000C077F401C078F402C079F403C0E2
:1014CC007AF46AC400F06BC401F06CC402F06DC411
:1014DC0003F077C404F078C405F079C406F07AC43C
:1014EC0007F037EC05F000C072F401C073F402C0D1
:1014FC0074F403C075F45BC400F00FEC04F072C418
:10150C0004F073C405F074C406F075C407F098ECCD
:10151C0001F0CAEC05F000C076F476C468F46EC431
:10152C0000F06FC401F070C402F071C403F077C412
:10153C0004F078C405F079C406F07AC407F037ECEF
:10154C0005F000C072F401C073F402C074F403C05F
:10155C0075F45CC400F00FEC04F072C404F073C4B6
:10156C0005F074C406F075C407F098EC01F0CAECF1
:10157C0005F000C069F4600E765D11E2400E695D05
:10158C000EE2000E685D0BE3000E695D08E368C4B3
:10159C007BF469C47CF45FC47DF4A4EC06F0602B8E
:0415AC0080D71200D2
:1015B000086A080E0C6E003408360450085ED8B075
:0E15C00002D00826D89000360C2EF5D7120067
:1015CE00086A096A100E0C6E01340836093604508A
:1015DE00085E0550D8A0053C095ED8B007D004506F
:1015EE0008260550D8B0053C0926D890003601369D
:0615FE000C2EEAD71200DA
:101604005BC45DF4200E04015B5D01E237D05D51E3
:101614007F0801E233D05E6B050E5E5D2CE2200E86
:101624005D5D006E050E0002F3CF00F05E510026F2
:10163400016A000E0122340E0024F66E3F0E0120D2
:10164400F76E000EF86E000E01BEFF0EF8220900C0
:10165400F5CF00F000C05FF400C07BF4DAEC04F0D6
:1016640004015C51000804E25FC47BF4DAEC04F08A
:0E16740004015E2BD1D77B6BDAEC04F0120080
:10168200200E04015B5D04E35B517F0801E301D09E
:1016920033D0050E5B03F3CF5CF4F4CF5DF4A00E00
:1016A2005C5F000E5D5B050E5E6F000E5F6F800E6D
:1016B200006E800E5F19005C02E15E51000819E2C3
:1016C200340E5C25F66E3F0E5D21F76E000EF86E4D
:1016D200000E5DBFFF0EF8220900F5CF7BF4DAECB5
:1016E20004F004015C4B5D2B010E5E5F000E5F5B3C
:0A16F200DED77B6BDAEC04F0120087
:1016FC000900F5CFE6FF0006FBE10106F9E1120057
:10170C00860ED56E0B0ED76EDC0ED66EF294306A4A
:06171C00316AF28A12009E
:101722000101446B456B000E455D02E1800E445D94
:1017320012E2A10E4425E16E000E4521E26EE66A38
:10174200010E4425006E000E4521016E00C044F1D9
:1017520001C045F1E8D7AECF40F10001A16B010114
:10176200406B446B456B3D6B3E6B2C6A2D6A9D8AC8
:02177200120063
:1017740004014F05516F4E05006E070E0016400E12
:1017840000107B6F27EC05F02B50010A0DE1050ECC
:1017940004015103F3CF00F07F0E0016800E0010F9
:1017A4007B6F27EC05F00CD0060E04015103F3CF38
:1017B40000F07F0E0016800E00107B6F27EC05F002
:0817C40050C45BF45CDF12006D
:1017CC0004014F05516F4E05006E070E0016400EBA
:1017DC0000107B6F27EC05F02DD051C400F00036C3
:1017EC000090003600907F0E0016800E0010040151
:1017FC007B6F27EC05F028D0060E04015103F3CFC4
:10180C0000F07F0E0016800E00107B6F27EC05F0A9
:10181C001BD051C400F0003600900036009000360A
:10182C0000907F0E0016800E001004017B6F27ECD9
:10183C0005F00AD004015051010ACFE05051020AC0
:0A184C00DBE05051030AE5E0120052
:1018560004014F05536F4E05006E070E0016400E2D
:1018660000107B6F27EC05F0060E04015303F3CF3F
:1018760000F07F0E0016800E00107B6F27EC05F03F
:1018860004014E51080801E222D050C4F6FF51C4AB
:10189600F7FF52C4F8FF0900F5CF01F00150000828
:1018A60016E25351100801E212D050C4F6FF51C49B
:1018B600F7FF52C4F8FF0900F5CF5BF4010E50277D
:1018C600000E51235223DADE0401532BDED7120019
:1018D60004017B6BDAEC04F0060E04017B6FDAEC94
:1018E60004F0090E04017B6FDAEC04F0090E040122
:1018F6007B6FDAEC04F0060E04017B6FDAEC04F081
:1019060004017B6BDAEC04F004017B6BDAEC04F087
:0A19160004017B6BDAEC04F0120010
:101920004EC402F04FC403F002C000F003C001F047
:10193000024A032A00C0E9FF01C0EAFFEE5201E0BB
:10194000F3D704014E51025C006E4F510358016EF3
:0A195000010E005E000E015A1200A5
:10195A00070E04014F15006E400E00107B6F27EC36
:10196A0005F07F0E04014E15006E800E00107B6F8D
:06197A0027EC05F012004D
:101980004EC4F6FF4FC4F7FF50C4F8FF0900F5CF6F
:1019900051F404015151000815E24EC4F6FF4FC442
:1019A000F7FF50C4F8FF0900F5CF00F000C051F474
:1019B000010E4E27000E4F23502300C05BF497EC1E
:0619C00007F0E7D712005A
:1019C6002E0E0101276F0F0E286F5B0E296F040E76
:1019D6002A6F1E0E2F6F1A0E306F000E316F000E1B
:1019E600326FFF0E396FFF0E3A6F000E3B6F000E1F
:1019F6003C6FFF0E356FFF0E366F000E376F000E11
:101A0600386FAC8A900EAB6E948E949C9EAA03D0CF
:081A1600AECF00F0FBD7120077
:101A1E00AECF01F0ABA202D0AB98AB8801C000F004
:021A2E001200A4
:101A30004EC450F44FC451F450C45BF451C45CF430
:101A400027EC08F000C052F4000E0401536F000EA2
:101A5000531902E1000E521901E121D0800E030A50
:101A6000006E800E5119005C02E15051FF0801E246
:101A700016D052C45BF497EC07F01A0E0C6EF80EF9
:101A80000D6E0D2EFED70C2EFCD700000401504B1E
:101A9000512B000E531902E1000E5219CDE1120034
:101AA000806A0F01386B388138832F0E926E9298BE
:101AB000898892868086396BFF0E816EFF0E936E49
:101AC0009380938293849386796A786A8B6A826A18
:0A1AD0003A6B800E946E606A1200FB
:101ADA008B848B808B94050E0B6E0F0E0C6EF10EA1
:101AEA000D6E0D2EFED70C2EFCD70B2EFAD78B843B
:101AFA00210E04017B6F27EC05F0900E04017B6F29
:101B0A0027EC05F0050E04017B6F27EC05F0130E98
:101B1A0004017B6F27EC05F0200E04017B6F27EC94
:101B2A0005F0340E0C6EF10E0D6E0D2EFED70C2E36
:101B3A00FCD7000000000C0E04017B6F27EC05F0B7
:101B4A0031EC08F0030E0B6E080E0C6E770E0D6E5C
:101B5A000D2EFED70C2EFCD70B2EFAD7400E040101
:101B6A007B6F27EC05F0800E04017B6F27EC05F0F4
:021B7A00120057
:101B7C000401516B030E515D0AE251514F25E16E88
:101B8C00000E5021E26E200EE66E512BF3D7515110
:101B9C004F25E16E000E5021E26EE66A510751515D
:101BAC004F25526F000E5021536F0A0E046E4EC417
:101BBC0000F0F8DC08C000F0300E002652C4E1FF43
:101BCC0053C4E2FF00C0E6FF0A0E046E4EC400F0E0
:101BDC00E9DC00C04EF40050000A01E102D05107CC
:041BEC00DED712002E
:101BF0000D0E04015B6F97EC07F00A0E04015B6F9A
:061C000097EC07F0120052
:101C060004014F05526F4E05006E070E0016400E7A
:101C160000107B6F27EC05F0050E04015203F3CF8D
:101C260000F07F0E0016800E00107B6F27EC05F08B
:101C360004014E51080801E217D050C4E9FF51C40F
:101C4600EAFFEE50000810E25251100801E20CD0F3
:101C560050C4E9FF51C4EAFFEECF5BF4504B512B61
:0A1C66000DDD0401522BE9D7120036
:101C70004EC45BF44FC45CF450C45DF44FC45EF4D6
:101C800052C45FF486EC09F04EC45BF451C45CF4BA
:101C900050C45DF451C45EF452C45FF486EC09F0A4
:101CA00050C45BF44FC45CF450C45DF451C45EF4A2
:101CB00052C45FF486EC09F04EC45BF44FC45CF48C
:101CC0004EC45DF451C45EF452C45FF486EC09F076
:021CD000120000
:101CD2000401516B4EC4E9FF4FC4EAFFEECF50F44A
:101CE2005051000A0FE050C45BF497EC07F0040176
:101CF200512B51514E25E96E000E4F21EA6EEECF67
:061D020050F4EED71200C0
:101D08004EC4E9FF4FC4EAFFEECF50F4000E0401C1
:101D1800516F000E516F000E511902E1200E50193B
:101D280007E0000E511902E1090E501901E003D035
:101D38004E4B4F2BE5D7526B536B546B556B000EC4
:101D4800511902E12D0E501905E1544B552B4E4BFC
:101D58004F2B08D0000E511902E12B0E501902E149
:101D68004E4B4F2B4EC4E9FF4FC4EAFFEECF50F461
:101D7800000E516F000E516F50C45BF49EEC07F0DB
:101D8800005219E052C400F053C401F00A0E046E68
:101D9800000E056EBAEC03F0300E505D026E000EB8
:101DA8005159036E02500024526F03500120536FA3
:101DB8004E4B4F2BD7D75451551108E052510008BC
:101DC800006E53C401F0000E015604D052C400F056
:061DD80053C401F01200EB
:101DDE000401526B050E525D0AE252515025E16E1E
:101DEE00000E5121E26E200EE66E522BF3D75251A9
:101DFE005025E16E000E5121E26EE66A52075251F5
:101E0E005025536F000E5121546F0A0E046E000EB2
:101E1E00056E4EC400F04FC401F0E7EC0AF008C0A6
:101E2E0000F009C001F0300E002653C4E1FF54C487
:101E3E00E2FF00C0E6FF0A0E046E000E056E4EC4F1
:101E4E0000F04FC401F0E7EC0AF000C04EF401C000
:101E5E004FF4000E011802E1000E001801E102D04D
:061E6E005207CDD712005F
:101E74000B6A0350D8B480EF0FF002500A6E028E42
:101E84008E0E035E03AE84EF0FF0036C080E035C4A
:101E9400D8A05FEF0FF0036E013602C001F0026AB2
:101EA400080E035CD8A05FEF0FF0036E0136016AE1
:101EB4000350D8A4D89069EF0FF00350D8B469EF59
:101EC4000FF0D89002320132032E63EF0FF00BBCF7
:101ED40001A076EF0FF0D8A076EF0FF0012AD8B466
:101EE400022A02BE93EF0FF00AAE99EF0FF0021E22
:101EF400011E012AD8B4022A99EF0FF0026A016A7E
:101F040099EF0FF00B800BAE9DEF0FF0026A0AAE53
:101F14009DEF0FF0FF0E026E016E0A3602329DEF46
:101F24000FF0010E0C6EA8EC03F09FEF0FF0000E03
:101F34000C6E9FEF0FF0FF0E0C6E0150006E0250FE
:041F4400016E120018
:101F480050C4F6FF51C4F7FF52C4F8FF0900F5CF9B
:101F580000F0005218E050C4F6FF51C4F7FF52C415
:101F6800F8FF0900F5CF00F04EC4E1FF4FC4E2FFCF
:101F780000C0E6FF04014E4B4F2B010E5027000E08
:101F880051235223DDD74EC4E1FF4FC4E2FFE66A76
:021F9800120035
:101F9A00040150510108516F526B000E525B010E41
:101FAA00576F000E586FFE0E006EFF0E016E50C482
:101FBA0004F0000E056EBAEC03F000C053F401C041
:101FCA0054F4596B5A6B50C455F4000E566F4EC4F4
:101FDA007BF450514F257C6F010E7D6FA4EC06F007
:101FEA004EC47BF450514F5D7C6F010E7D6FA4ECA3
:101FFA0006F050514E257B6F4FC47CF4010E7D6F65
:10200A00A4EC06F050514E5D7B6F4FC47CF4010E78
:10201A007D6FA4EC06F0800E5A19006E800E5619D8
:10202A00005C02E15551595DD8B07CD0800E52193E
:10203A00006E800E005C02E1000E515D12E3010E9B
:10204A00555F000E565B020E5325006E000E54219A
:10205A00016E00C053F401C054F4005051270150DE
:10206A005223594B5A2B020E5725006E000E582147
:10207A00016E00C057F401C058F4005051270150B6
:10208A00522359514E257B6F55514F257C6F010EB6
:10209A007D6FA4EC06F059514E5D7B6F55514F256B
:1020AA007C6F010E7D6FA4EC06F059514E257B6FB3
:1020BA0055514F5D7C6F010E7D6FA4EC06F05951AE
:1020CA004E5D7B6F55514F5D7C6F010E7D6FA4ECA9
:1020DA0006F055514E257B6F59514F257C6F010EE5
:1020EA007D6FA4EC06F055514E5D7B6F59514F251B
:1020FA007C6F010E7D6FA4EC06F055514E257B6F67
:10210A0059514F5D7C6F010E7D6FA4EC06F055515D
:10211A004E5D7B6F59514F5D7C6F010E7D6FA4EC54
:06212A0006F079D7120057
:10213000FF0E01012B6FFF0E2C6FFF0E2D6FFF0E98
:102140002E6FC26A2A1C006E0050C1160F0EC012FC
:06215000C08EC2801200E7
:10215600400E04017B6F27EC05F0800E04017B6FB7
:1021660027EC05F00401536B546B800E5419006E76
:10217600800E005C02E1400E535DD8B07BD0516BFF
:10218600526B800E5219006E800E005C02E10C0E3E
:10219600515D63E253C400F054C401F00C0E046EAA
:1021A600000E056EBAEC03F0515100265251012281
:1021B60000C057F401C058F400504E25F66E015089
:1021C6004F21F76E000E5021F86E0900F5CF5AF434
:1021D600800E596F556B566B595100083BE2030E42
:1021E600006E51C457F452C458F4005005E05737F6
:1021F60057915837FF0FFAD755515727565158233D
:1022060059515A15016E015059190EE12A0E5B6F8C
:1022160097EC07F057C47BF453C47CF4010E040119
:102226007D6FA4EC06F00CD0200E5B6F97EC07F0E8
:1022360057C47BF453C47CF404017D6BA4EC06F014
:102246005933599F554B562B1A0E0D6E0D2EFED730
:102256000000C2D7514B522B94D70D0E5B6F97ECF3
:1022660007F00A0E04015B6F97EC07F00401534B6D
:06227600542B7BD712007F
:10227C00400E04017B6F27EC05F0800E04017B6F90
:10228C0027EC05F004014E6B4F6B800E4F19006E5E
:10229C00800E020A005C02E1FF0E4E5D0EE2480E5B
:1022AC004E25E96E010E4F21EA6EEECF7BF4DAEC8F
:1022BC0004F004014E4B4F2BE8D7400E7B6F27ECFC
:0E22CC0005F0800E04017B6F27EC05F0120078
:1022DA004EC400F04FC401F071EC09F0000E046E18
:1022EA00000E056E400E066E850E076E37EC05F081
:1022FA00000E046E000E056E000E066E890E076E45
:10230A001DEC04F000C04AF401C04BF402C04CF4C6
:10231A0003C04DF403EC09F000C054F401C055F4B5
:10232A00800E006E800E04015119005C02E15051CA
:10233A00000839E2800E5119006E800E005C02E13D
:10234A00090E505D30E25005006E070E0016400E71
:10235A0000107B6F27EC05F00401526B536B000EE3
:10236A00535D02E15F0E525D1EE2800E52117B6FD9
:10237A0027EC05F004015351555D02E15251545DB9
:10238A0005E33C0E7B6FDAEC04F004D004017B6BAE
:10239A00DAEC04F0060E0D6E0D2EFED700000401D5
:1023AA00524B532BDCD7400E7B6F27EC05F0800E87
:0A23BA0004017B6F27EC05F0120010
:1023C400400E04017B6F27EC05F0800E04017B6F47
:1023D40027EC05F004014E6B4F6B800E4F19006E15
:1023E400800E020A005C02E1FF0E4E5D0AE2480E16
:1023F4004E25E16E010E4F21E26EE66A4E4B4F2BE5
:10240400ECD7400E7B6F27EC05F0800E04017B6F48
:0624140027EC05F01200A8
:10241A0004014E05006E070E0016400E00107B6F79
:10242A0027EC05F0060E04014F03F3CF00F07F0EF0
:0E243A000016800E00107B6F27EC05F01200DC
:10244800C26A2A1C006E0050C1160F0EC012C08E40
:102458004EC400F000360090003600900050C212C2
:10246800C280FEEC08F0C282C2A201D0FDD7C4CF60
:1024780001F0006A00C04FF401C050F4C3500012CC
:10248800000E011200C04FF401C050F4C290000EBB
:102498000014026E0150800B036E000E031802E157
:1024A800000E021803E004014F6B506B4FC400F09C
:0624B80050C401F0120007
:1024BE000401566B046A056A066A076A4EC400F088
:1024CE004FC401F050C402F051C403F03DEC06F0CD
:1024DE00010ED8B0000E006E005203E0507F010EC8
:1024EE00566F4EC400F04FC401F050C402F051C4F8
:1024FE0003F0830E046EF90E056E220E066E7C0E30
:10250E00076E37EC05F000C04EF401C04FF402C068
:10251E0050F403C051F400C05BF401C05CF402C07F
:10252E005DF403C05EF467EC08F000C004F001C077
:10253E0005F002C006F003C007F04EC400F04FC411
:10254E0001F050C402F051C403F017EC06F0000E77
:10255E00046E000E056E000E066E810E076E37ECD1
:10256E0005F000C04EF401C04FF402C050F403C099
:10257E0051F400C004F001C005F002C006F003C023
:10258E0007F0000E006E000E016E000E026E800E41
:10259E00036E3DEC06F0010ED8B0000E006E005238
:1025AE0020E0000E046E000E056E000E066E800E0C
:1025BE00076E4EC400F04FC401F050C402F051C477
:1025CE0003F017EC06F000C04EF401C04FF402C049
:1025DE0050F403C051F404015653010ED8A4000E5A
:1025EE00566F4EC404F04FC405F050C406F051C4EB
:1025FE0007F0000E006E000E016E000E026E7F0ED2
:10260E00036E3DEC06F0010ED8B0000E006E0052C7
:10261E001AE04EC404F04FC405F050C406F051C485
:10262E0007F0000E006E000E016E000E026E800EA0
:10263E00036E17EC06F000C04EF401C04FF402C05A
:10264E0050F403C051F404014EC400F04FC401F025
:10265E0050C402F051C403F04EC404F04FC405F050
:10266E0050C406F051C407F037EC05F000C052F428
:10267E0001C053F402C054F403C055F400C05BF41F
:10268E0001C05CF402C05DF403C05EF4D50E5F6F52
:10269E00420E606F000E616F040E626F000E636F6C
:1026AE00AAEC07F04EC404F04FC405F050C406F077
:1026BE0051C407F037EC05F000C04EF401C04FF4E2
:1026CE0002C050F403C051F452C45BF453C45CF422
:1026DE0054C45DF455C45EF4260E5F6F440E606FF5
:1026EE00000E616F030E626F000E636FAAEC07F0AF
:1026FE0000C004F001C005F002C006F003C007F0F0
:10270E004EC400F04FC401F050C402F051C403F0A7
:10271E001DEC04F000C04EF401C04FF402C050F4A2
:10272E0003C051F4040156530DE0000E4E19006E15
:10273E00000E4F19016E800E5019026E000E5119C7
:10274E00036E08D04EC400F04FC401F050C402F026
:06275E0051C403F012005B
:102764004EC4E9FF4FC4EAFFEE50000A12E04EC423
:10277400E9FF4FC4EAFFEECF5BF450C45CF402EC13
:102784000BF004014E4B4F2B0D0E0D6E0D2EFED78C
:04279400E7D7120071
:1027980041EC22F0700ED36E9B6A9B9C50EC0DF0BE
:1027A8000401486B496B000E495D02E1800E485DEB
:1027B8000AE2A10E4825E16E000E4921E26EE66AA2
:1027C800484B492BF0D7486B496B000E495D02E135
:1027D800180E485D0AE2890E4825E16E000E49216F
:1027E800E26EE66A484B492BF0D7486B496B000EFE
:1027F800495D02E1500E485D0AE2390E4825E16E56
:10280800000E4921E26EE66A484B492BF0D7486B27
:10281800496B390E0101216F000E226F8998B88625
:10282800B06ACF0EAF6EAC84E3EC0CF00C0E040172
:102838005B6F97EC07F00B0E0B6E260E0C6E5D0EA1
:102848000D6E0D2EFED70C2EFCD70B2EFAD70000DE
:102858000000370E04014E6F430E4F6F000E506F8D
:10286800C0EC0CF04F0E04014E6F410E4F6F000E7E
:10287800506FC0EC0CF0B10E04014E6F410E4F6F5B
:10288800000E506FC0EC0CF0150E0B6E4B0E0C6E5C
:10289800BE0E0D6E0D2EFED70C2EFCD70B2EFAD7C2
:1028A8000000390E0101216F000E226F04014E6BEA
:1028B8004F6B18EC0DF0040E4E6F440E4F6F000E68
:1028C800506FC0EC0CF0150E0B6E4B0E0C6EBE0E5E
:1028D8000D6E0D2EFED70C2EFCD70B2EFAD700004E
:1028E800F8EC0DF02B6A6DEC0DF08998200E0401C0
:1028F8004E6F000E4F6F18EC0DF0290E0B6E960EF2
:102908000C6E7F0E0D6E0D2EFED70C2EFCD70B2EE7
:10291800FAD7010E4E6F010E4F6FD10E506F430E56
:10292800516F000E526F2BEC0CF0030E0B6E080E5D
:102938000C6E770E0D6E0D2EFED70C2EFCD70B2EBF
:10294800FAD780A6EFD331EC08F0200E0101256FED
:10295800010E0401486F000E496F000E495D02E147
:10296800080E485D26E2010E0101236F000E246F58
:10297800000E245D02E1110E235D17E248C44EF4F7
:1029880023C14FF425C150F4BAEC0BF00101252BFB
:10299800340E0C6EF10E0D6E0D2EFED70C2EFCD7DC
:1029A80000000000234B242BE3D70401484B492B9C
:1029B800D4D7520E0B6E2B0E0C6E000E0D6E0D2E14
:1029C800FED70C2EFCD70B2EFAD7000031EC08F0FE
:1029D800010E04014E6F010E4F6F9E0E506F430E95
:1029E800516F000E526F2BEC0CF0020E4E6F010E61
:1029F8004F6F690E506F440E516F000E526F2BECE3
:102A08000CF0030E4E6F010E4F6F27C050F428C014
:102A180051F429C052F42BEC0CF0040E4E6F010E49
:102A28004F6FAF0E506F430E516F000E526F2BEC6D
:102A38000CF0050E4E6F010E4F6F5A0E506F430E7D
:102A4800516F000E526F2BEC0CF0060E4E6F010EFC
:102A58004F6F6B0E506F430E516F000E526F2BEC81
:102A68000CF0070E4E6F010E4F6F150E506F440E8F
:102A7800516F000E526F2BEC0CF0080E4E6F010ECA
:102A88004F6FE20E506F430E516F000E526F2BECDA
:102A98000CF0290E0B6E960E0C6E7F0E0D6E0D2E21
:102AA800FED70C2EFCD70B2EFAD731EC08F0140EFB
:102AB80004014E6F410E4F6F000E506FC0EC0CF0CA
:102AC800620E04014E6F420E4F6F000E506FC0EC45
:102AD8000CF0010E2B6E31EC08F00101236B246B16
:102AE800000E245D02E1080E235D42E22351010F2E
:102AF80004014E6F010E4F6F020E506FE6EC0BF0A3
:102B08000401486B496B000E495D02E1130E485DF4
:102B18001EE201012351010F04014E6F48C44FF416
:102B28000A0E046E000E056E48C400F049C401F098
:102B3800E7EC0AF008C000F009C001F0300E0024EC
:102B4800506FBAEC0BF00401484B492BDCD7020E4E
:102B58000B6E040E0C6EBA0E0D6E0D2EFED70C2EDB
:102B6800FCD70B2EFAD700000101234B242BB8D732
:102B78003D0E0B6EE10E0C6E3F0E0D6E0D2EFED748
:102B88000C2EFCD70B2EFAD7000000002B6A270E5C
:102B980004014E6F420E4F6F000E506FC0EC0CF0E8
:102BA800940E04014E6F420E4F6F000E506FC0EC32
:102BB8000CF031EC08F002DC340E04014E6F390ED3
:102BC8004F6F000E506FABEC10F03EEC11F01F0E83
:102BD8000B6E710E0C6E1E0E0D6E0D2EFED70C2E8A
:102BE800FCD70B2EFAD7000031EC08F0E2EC11F01C
:102BF800340E04014E6F3C0E4F6F000E506FABEC5D
:102C080010F03EEC11F01F0E0B6E710E0C6E1E0EC6
:102C18000D6E0D2EFED70C2EFCD70B2EFAD700000A
:102C2800F8EC0DF0030E04014E6F420E4F6F000ECC
:102C3800506FC0EC0CF031EC08F0E2EC11F004013C
:102C4800486B496B000E495D02E15F0E485D41E249
:102C58000101235104014825006E0101245104019A
:102C68004921016E71EC09F0D00E046E0F0E056E4D
:102C7800490E066E800E076E37EC05F0000E046EE6
:102C8800000E056E700E066E830E076E1DEC04F0C6
:102C980000C04EF401C04FF402C050F403C051F418
:102CA8000ADC000E046E000E056E700E066E830EB2
:102CB800076E37EC05F03AEC0FF00050200F7C6FF0
:102CC80048C47BF4010E7D6FA4EC06F0484B492BF9
:102CD800B9D73EEC11F0290E0B6E960E0C6E7F0ED6
:102CE8000D6E0D2EFED70C2EFCD70B2EFAD7C00E6C
:102CF80004014E6F420E4F6F000E506FC0EC0CF087
:102D0800E2EC11F00401486B496B000E495D02E1E9
:102D1800410E485D10E25B6B48C45CF4600E5D6F69
:102D280048C45EF4010E5F6F86EC09F0080E482770
:102D3800000E4923EAD7486B496B000E495D02E152
:102D4800600E485D10E248C45BF45C6B48C45DF4F7
:102D5800400E5E6F010E5F6F86EC09F00C0E48277F
:102D6800000E4923EAD73EEC11F0290E0B6E960EA1
:102D78000C6E7F0E0D6E0D2EFED70C2EFCD70B2E73
:102D8800FAD7E2EC11F0240E04014E6F430E4F6F98
:102D9800000E506FC0EC0CF031EC08F0E2EC11F0D2
:102DA800010E04015B6F010E5C6F600E5D6F400EDB
:102DB8005E6F010E5F6F86EC09F0010E5B6F400ECF
:102DC8005C6F600E5D6F010E5E6F010E5F6F86ECCB
:102DD80009F0300E5B6F010E5C6F300E5D6F400EB8
:102DE8005E6F010E5F6F86EC09F0010E5B6F200EBF
:102DF8005C6F600E5D6F200E5E6F010E5F6F86EC7C
:102E080009F03EEC11F0290E0B6E960E0C6E7F0E3B
:102E18000D6E0D2EFED70C2EFCD70B2EFAD7E2EC3A
:102E280011F031EC08F0DF0E04014E6F410E4F6FC8
:102E3800000E506FC0EC0CF0890E04014E6F000EAE
:102E48004F6F7A0E506F440E516F000E526FA4EC04
:102E58000FF0890E04014E6F000E4F6F84EC0EF0D8
:102E680000C037F001C038F000C04EF401C04FF484
:102E7800890E506F000E516FEFEC0EF0010E4E6F81
:102E8800030E4F6F890E506F000E516F03EC0EF05A
:102E980037C04EF438C04FF4020E506F000E516F19
:102EA8006DEC11F0050E0B6E0F0E0C6EF10E0D6E23
:102EB8000D2EFED70C2EFCD70B2EFAD7890E040147
:102EC8004E6F000E4F6F7E0E506F440E516F000E06
:102ED800526FA4EC0FF0890E04014E6F000E4F6F75
:102EE80084EC0EF000C037F001C038F000C04EF49A
:102EF80001C04FF4890E506F000E516FEFEC0EF0C9
:102F0800040E4E6F030E4F6F890E506F000E516FF7
:102F180003EC0EF037C04EF438C04FF4050E506F76
:102F2800000E516F6DEC11F0050E0B6E0F0E0C6E4E
:102F3800F10E0D6E0D2EFED70C2EFCD70B2EFAD7E8
:102F4800890E04014E6F000E4F6F700E506F440EC5
:102F5800516F000E526FA4EC0FF0890E04014E6FF2
:102F6800000E4F6F84EC0EF000C037F001C038F04F
:102F780000C04EF401C04FF4890E506F000E516F1F
:102F8800EFEC0EF0890E4E6F000E4F6F69EC0EF0ED
:102F9800F8EC0DF0070E04014E6F030E4F6F890E0B
:102FA800506F000E516F03EC0EF037C04EF438C06E
:102FB8004FF4080E506F000E516F6DEC11F0290E92
:102FC8000B6E960E0C6E7F0E0D6E0D2EFED70C2E10
:102FD800FCD70B2EFAD7360E04014E6F440E4F6FF6
:102FE800000E506FC0EC0CF031EC08F0E2EC11F080
:102FF800010E04014E6F010E4F6F5F0E506F3F0EB2
:10300800516F010E526F38EC0EF0080E4E6F080E1D
:103018004F6F500E506F380E516F010E526F38ECD3
:103028000EF0100E4E6F100E4F6F480E506F300E90
:10303800516F010E526F38EC0EF03EEC11F0290E74
:103048000B6E960E0C6E7F0E0D6E0D2EFED70C2E8F
:10305800FCD70B2EFAD7FD0E04014E6F420E4F6FB0
:10306800000E506FC0EC0CF0E2EC11F0300E0401D1
:103078004E6F200E4F6F1E0E506FCDEC0FF0300EBE
:103088004E6F200E4F6F140E506FCDEC0FF0300EB8
:103098004E6F200E4F6F0A0E506FCDEC0FF0300EB2
:1030A8004E6F200E4F6F050E506FCDEC0FF0080ECF
:1030B8004E6F080E4F6F040E506FCDEC0FF0580E88
:1030C8004E6F380E4F6F040E506FCDEC0FF03EEC84
:1030D80011F0330E0B6EBB0E0C6EDF0E0D6E0D2E47
:1030E800FED70C2EFCD70B2EFAD70000000031ECCF
:1030F80008F0060E04014E6F010E4F6F7C0E506FE4
:10310800430E516F000E526F2BEC0CF0290E0B6E14
:10311800960E0C6E7F0E0D6E0D2EFED70C2EFCD764
:103128000B2EFAD780B614D0010E4E6F010E4F6FDA
:10313800490E506F430E516F000E526F2BEC0CF07E
:10314800810E4E6F410E4F6F000E506FC0EC0CF0A9
:103158007C0E04014E6F420E4F6F000E506FC0EC94
:103168000CF098EC10F0AB0E04014E6F420E4F6F4E
:10317800000E506FC0EC0CF031EC08F0F28CF28EBF
:10318800010E196E000E1A6E010E04014E6F010E2B
:103198004F6FC00E506F430E516F000E526F2BECE5
:1031A8000CF019C04EF41AC04FF4890E506F000E7F
:1031B800516FEFEC0EF0010E4E6F090E4F6F890E36
:1031C800506F000E516F03EC0EF0460E4E6F440E1A
:1031D8004F6F000E506FC0EC0CF0890E04014E6F5B
:1031E800000E4F6F69EC0EF0020E4E6F010E4F6F1E
:1031F8008D0E506F430E516F000E526F2BEC0CF07A
:103208004E6B24EC12F000C02EF001C02FF000C06D
:103218004EF401C04FF4890E0401506F000E516F37
:10322800EFEC0EF0020E4E6F040E4F6F0DEC12F025
:10323800890E04014E6F000E4F6F010E506FB2ECF5
:1032480013F0020E04014E6F0E0E4F6F0DEC12F0CC
:103258006BEC0CF0020E04014E6F0F0E4F6F0DEC6D
:1032680012F0430E04015B6F41EC0BF0500E0401A9
:103278004E6F440E4F6F000E506FC0EC0CF0890E6D
:1032880004014E6F000E4F6F69EC0EF0F8EC0DF074
:1032980086EC0BF091EC0BF0000E2D1802E1000EFD
:1032A8002C1807E1000E311802E1000E301801E178
:1032B800F3D7000E311802E1000E3018D8A432D32B
:1032C800750E04014E6F440E4F6F000E506FC0EC28
:1032D8000CF031EC08F0030E0B6E080E0C6E770E36
:1032E8000D6E0D2EFED70C2EFCD70B2EFAD7A10E85
:1032F80004014E6F000E4F6F90EC0CF000C037F0D9
:1033080001C038F0A10E4E6F000E4F6F69EC0EF041
:10331800A10E356E000E366EA10E336E000E346EA1
:1033280033C0E9FF34C0EAFFEE50410AD8A4E6D022
:10333800010E3324E96E000E3420EA6EEE50540A72
:10334800D8A4DCD0030E3324E96E000E3420EA6ED4
:10335800EE502C0A17E1030E3324E16E000E3420E0
:10336800E26EE66A020E3324E96E000E3420EA6E3D
:10337800300EEE5C016E01C032F00150080802E226
:10338800010E326E060E3324E96E000E3420EA6E0A
:10339800EE502C0AD8A4B2D0060E3324E16E000EEB
:1033A8003420E26EE66A040E3324006E000E3420E8
:1033B800016E00C033F001C034F000C04EF401C00B
:1033C8004FF484EC0EF000C026F1010E005C05E31A
:1033D80001012651100801E303D00101010E266FF7
:1033E800070E3524006E000E3620016E00C035F041
:1033F80001C036F000C04EF401C04FF490EC0CF060
:1034080000C037F001C038F0040E026E00C041F170
:1034180001C042F1025006E0010142334133429FAC
:10342800FF0FF9D70101414B422B04014E6B4F6B43
:10343800ADEC0CF00401486B496B010142510401E9
:10344800495D04E1010141510401485D57E2100E54
:103458003524006E000E3620016E00C0E9FF01C061
:10346800EAFFEECF40F100C0E1FF01C0E2FFE66AEB
:1034780048510101262504014E6F32C04FF435C072
:1034880050F436C051F403EC0EF048C44EF449C46D
:103498004FF4890E506F000E516FEFEC0EF0890E4D
:1034A8004E6F000E4F6F69EC0EF0090E5B6F97ECD4
:1034B80007F0A10E04014E6F000E4F6F69EC0EF07D
:1034C800F8EC0DF0050E0B6E0F0E0C6EF10E0D6E76
:1034D8000D2EFED70C2EFCD70B2EFAD7100E352446
:1034E800E16E000E3620E26E40C1E6FF100E352672
:1034F800000E36220401484B492B9FD733C0E9FF01
:1035080034C0EAFFEE50500AD8A477D0010E332415
:10351800E96E000E3420EA6EEE50490A6EE1040EA0
:103528003324E96E000E3420EA6EEE502C0A65E171
:10353800040E3324E16E000E3420E26EE66A020EB9
:103548003324006E000E3420016E00C033F001C039
:1035580034F000C04EF401C04FF484EC0EF000C00B
:1035680026F1010E005C05E3010126515F0801E325
:1035780003D00101010E266F030E3324006E000EE6
:103588003420016E00C033F001C034F000C04EF4A6
:1035980001C04FF484EC0EF000C032F0010E005C64
:1035A80004E332503F0801E302D0010E326E360EBA
:1035B800AD6EE2EC11F026C17BF432C07CF4010E52
:1035C80004017D6FA4EC06F03EEC11F00B0E0B6EBF
:1035D800260E0C6E5D0E0D6E0D2EFED70C2EFCD732
:1035E8000B2EFAD700000000590E04014E6F440E4E
:1035F8004F6F000E506FC0EC0CF033C0E9FF34C0C1
:10360800EAFFEE50520AD8A418D1010E3324E96E0D
:10361800000E3420EA6EEE50450AD8A40ED1040EEE
:103628003324E96E000E3420EA6EEE502C0AD8A43A
:1036380004D1040E3324E16E000E3420E26EE66AF3
:10364800070E3324E16E000E3420E26EE66A0A0E9D
:103658003324E16E000E3420E26EE66A0D0E332448
:10366800E16E000E3420E26EE66A020E3524006E2A
:10367800000E3620016E00C033F001C034F000C0E7
:103688004EF401C04FF484EC0EF000C03FF1010E7F
:10369800005C05E301013F515F0801E303D001012C
:1036A800010E3F6F050E3524006E000E3620016EA8
:1036B80000C033F001C034F000C04EF401C04FF434
:1036C80084EC0EF000C043F1010E005C05E301013B
:1036D80043513F0801E303D00101010E436F080E77
:1036E8003524006E000E3620016E00C033F001C094
:1036F80034F000C04EF401C04FF484EC0EF000C06A
:1037080047F1010E005C05E3010147515F0801E341
:1037180003D00101010E476F0B0E3524006E000E19
:103728003620016E00C033F001C034F000C04EF402
:1037380001C04FF484EC0EF000C046F1010E005CAD
:1037480005E3010146513F0801E303D00101010EE1
:10375800466F3FC14EF4890E04014F6F000E506F43
:10376800BEEC0DF0890E4E6F000E4F6F69EC0EF037
:10377800090E5B6F97EC07F043C14EF4890E040104
:103788004F6F000E506FBEEC0DF0890E4E6F000E9D
:103798004F6F69EC0EF0090E5B6F97EC07F047C1AD
:1037A8004EF4890E04014F6F000E506FBEEC0DF001
:1037B800890E4E6F000E4F6F69EC0EF0090E5B6FAD
:1037C80097EC07F046C14EF4890E04014F6F000EC6
:1037D800506FBEEC0DF0890E4E6F000E4F6F69EC06
:1037E8000EF0F8EC0DF0360EAD6EE2EC11F03FC1C4
:1037F8004EF443C14FF447C150F446C151F4010E91
:103808000401526F38EC0EF03EEC11F00B0E0B6E0B
:10381800260E0C6E5D0E0D6E0D2EFED70C2EFCD7EF
:103828000B2EFAD700000000610E04014E6F440E03
:103838004F6F000E506FC0EC0CF033C0E9FF34C07E
:10384800EAFFEE50430A16E1010E3324E96E000E3A
:103858003420EA6EEE504C0A0DE1020E3324E96E74
:10386800000E3420EA6EEE50530A04E1E2EC11F047
:103878003EEC11F033C0E9FF34C0EAFFEE50420AD3
:1038880050E133C04EF434C04FF490EC0CF000C05B
:1038980037F001C038F0486B496B3850495D02E198
:1038A8003750485D14E248513324E96E49513420B9
:1038B800EA6EEE502C0A08E148513324E16E495172
:1038C8003420E26EE66A03D0484B492BE6D73850DD
:1038D800495D02E13750485D24E2010E33244E6F02
:1038E800000E34204F6F84EC0EF000C037F001C09A
:1038F80038F000C04EF401C04FF448513324006E34
:1039080049513420016E010E0024E96E000E012099
:10391800EA6E300EEE5C506F516B000E515B6DEC31
:0C39280011F002D0194A1A2A2FD4FFD740
:1044820010EE19F0130E006E010E016E110EF66E93
:0E449200430EF76E000EF86E7EEC0BF012007B
:103934000000000000000000000000000000000083
:103944000000000000000000000000000000000073
:103954000000000000000000000000000000000063
:103964000000000000000000000000000000000053
:103974000000000000000000000000000080300093
:103984000000000003F000000180F80000000000C7
:1039940003F800000181F0C00008000003FC0000EF
:1039A4000181C0C0001C0000061C0000018180C011
:1039B40000180000060C0000018300000000000055
:1039C400060C00000383000000000000060C000049
:1039D4000383000000000000060C1C10230FE0818C
:1039E40002080700061C7E18631FE1C186181F80A9
:1039F4000638FF38631FE1C386183FC00FF9E7306C
:103A0400630601C3061839C00FF1C630630601C34B
:103A1400061870C00FC18630E30601830E1860C01B
:103A24000C038630E70601830E3860C00C030630B1
:103A3400C60601830C3860C00C030630C606018339
:103A44000C38E0C01C030670C60E01870C38E180F8
:103A540018030670C60C01870C38E18018030E7039
:103A6400C60C01870C30638018039E7FC60C018747
:103A7400FC307F001803FE3FCE0C0183FC307E0037
:103A84000001F63FCC0C0383FC303C000000000036
:103A9400800C038008300000000000000008038050
:103AA4000030000000000000000023000630000089
:103AB4000000000000007300063000000000000059
:103AC40000003700076000000000000000003E0016
:103AD40003E000000000000000001E0003C000001E
:103AE4000000000000001C000180000000007800BD
:103AF400000000000003E0000000FC0000000000E3
:103B04000007E0000001F80000000000000FC00002
:103B14000003C00000000000001E0000000380003D
:103B240000000000001C00000007800000000000EE
:103B3400001C00000007608603800E00003D043076
:103B4400003FF1FF0FE07F8001FFCFF8007FF3FF1C
:103B54001FF0FFC001FFCFFC003FE3FF3CF1F3C0C7
:103B640001FF1FFC000F03E778F1C7C000781F387E
:103B7400000E038677E3DF8000781E38000E038092
:103B8400FFC3FE0000701C00000E0780FF03F80056
:103B940000701C00000E0780FC03E00000701C0095
:103BA400001E0700F023808000703C00001E070008
:103BB400FDF3E78000F03C00701C07007FE3FF8307
:103BC40080F03800F01C07003FC1FF0780E0380098
:103BD400601C02000E00380380E010000018000092
:103BE4000000000000400000000000000000000091
:103BF40000000000000000000000000000000000C1
:103C040000000000000000000000000000000000B0
:103C140000000000000000000000000000000000A0
:103C24000000000000000000000000000000000090
:103C3400FFFE2000000000000013FFFFFFFE200035
:103C4400000000000013FFFFFFFE20FF0001FFC083
:103C54000013FFFFFFFE20FF0001FFC00013FFFF62
:103C6400FFFE23FFE00FFFF80013FFFFFFFE23FF1B
:103C7400F03FFFFE0013FFFFFFFE230030FFFFFFB6
:103C8400C013FFFFFFFE230030FFFFFFC013FFFF41
:103C9400FFFE220033FFFFFFE013FFFFFFFE23FFC1
:103CA400E3FFFFFFE013FFFFFFFE23FFE7FFFFFF3C
:103CB400F013FFFFFFFE23FFE7FFFFFFF013FFFFFB
:103CC400FFFE21FFC7FFE3FFF813FFFFFFFE200005
:103CD4000FFFE1FFF813FFFFFFFE20000FFFC1FFFE
:103CE400F813FFFFFFFE20000FFFC1FFF813FFFFD3
:103CF400FFFE23C00FFFC1FFFC13FFFFFFFE23E005
:103D04000FFFC1FFFC13FFFFFFFE23FF0FFFC1FFE7
:103D1400FC13FFFFFFFE23FF0FFFC1FFFC13FFFF98
:103D2400FFFE23FF0FFFC1FFFC13FFFFFFFE23FF76
:103D34000FFFC1FFFC13FFFFFFFE20000FFFE1FF99
:103D4400FC13FFFFFFFE20000FFFE1FFFC13FFFF4A
:103D5400FFFE22010FFFFFFFFC13FFFFFFFE23E71F
:103D64000FFFFFFFFC13FFFFFFFE23EF0FFFFFFF1B
:103D7400FC13FFFFFFFE23EF0FFFFFFFFC13FFFF0A
:103D8400FFFE20FE0FFFFFFFFC13FFFFFFFE22FFDD
:103D94000FFFFFFFFC13FFFFFFFE23FF0FFFFFFFDB
:103DA400FC13FFFFFFFE23FF0FFFFFFFFC13FFFFCA
:103DB400FFFE23FF0FFFE0000013FFFFFFFE2200C2
:103DC4000FFFC0000013FFFFFFFE20000FFFC00025
:103DD4000013FFFFFFFE20000FFFC0000013FFFFD2
:103DE400FFFE223F0FFFC0FFFC13FFFFFFFE223F39
:103DF4000FFFC0FFFC13FFFFFFFE22FF0FFFC0FFFA
:103E0400FC13FFFFFFFE22FF0FFFC0FFFC13FFFFA9
:103E1400FFFE20000FFFC0FFFC13FFFFFFFE20008A
:103E24000FFFC0FFFC13FFFFFFFE23FF0FFFC0FFC8
:103E3400FC13FFFFFFFE23FF0FFFC0FFFC13FFFF78
:103E4400FFFE23FF0FFFC0FFFC13FFFFFFFE23FF56
:103E5400CFFFC0FFFC13FFFFFFFE22000FFFC0FFD8
:103E6400FC13FFFFFFFE22000FFFC0FFFC13FFFF48
:103E7400FFFE20000FFFE1FFF813FFFFFFFE23FF0B
:103E8400C7FFE1FFF813FFFFFFFE23FFE7FFF7FF84
:103E9400F813FFFFFFFE23FFE7FFF7FFF813FFFF11
:103EA400FFFE23FFE3FFFFFFF013FFFFFFFE2200EF
:103EB40003FFFFFFE013FFFFFFFE220001FFFFFFF0
:103EC400C013FFFFFFFE220001FFFFFFC013FFFF2F
:103ED400FFFE23FFF8FFFFFF0013FFFFFFFE23FF9A
:103EE400FC1FFFFE0013FFFFFFFE23FFFE07FFF88A
:103EF4000013FFFFFFFE23FFFE07FFF80013FFFF81
:103F0400FFFE2000000000000013FFFFFFFE200062
:103F1400000000000013FFFFFFFE2000000000006F
:103F24000023FFFFFFFE2000000000000023FFFF2E
:103F3400000000000000005F0000000700070014FC
:103F44007F147F14242A7F2A1223130864623649BB
:103F54005522500005030000001C224100004122AC
:103F64001C0014083E081408083E080800503000DD
:103F74000008080808080060600000201008040217
:103F84003E5149453E00427F40004261514946212D
:103F940041454B311814127F1027454545393C4A99
:103FA40049493001710905033649494936064949E9
:103FB400291E00363600000056360000081422413F
:103FC40000141414141400412214080201510906A7
:103FD400324979413E7E1111117E7F494949363E6D
:103FE400414141227F4141221C7F494949417F0986
:103FF4000909013E4149497A7F0808087F00417F49
:1040040041002040413F017F081422417F4040404D
:10401400407F020C027F7F0408107F3E4141413EF5
:104024007F090909063E4151215E7F091929464647
:104034004949493101017F01013F4040403F1F2070
:1040440040201F3F4038403F631408146307087042
:1040540008076151494543007F41410002040810AB
:10406400200041417F0004020102044040404040DE
:10407400000102040020545454787F4844443838E2
:1040840044444420384444487F3854545418087EE7
:104094000901020C5252523E7F0804047800447D08
:1040A40040002040443D007F1028440000417F40F0
:1040B400007C041804787C080404783844444438A8
:1040C4007C14141408081414187C7C08040408488C
:1040D40054545420043F4440203C4040207C1C2045
:1040E40040201C3C4030403C44281028440C505094
:1040F400503C4464544C44000836410000007F00A6
:104104000000413608001008081008784641467837
:104114007465737420224E6F6B69615F57726974A2
:10412400655F436861725F4154284C2C432C63687B
:1041340061722922206D6F646520384C20646520EB
:0B41440031382063617273200D0A0007
:10414F004D696B726F632070726F20372E31302084
:10415F0031384632364B3232205541525431204E8F
:10416F006F6B6961204C4344203936783634200A0E
:02417F000D0031
:104181000D0A2050696E205241353D3120646F6E19
:10419100632053414E532050726573656E74617490
:1041A100696F6E20737572204C434420200D0A0004
:1041B10050726F6A6574203A205465726D696E6140
:1041C1006C5F4E6F6B69615F387831365F313846AD
:0E41D10032364B32322E6D637070690D0A006B
:1041DF0054657374204261726772706168732061F5
:1041EF00766563203530302C3735302C3130303018
:0441FF00200D0A0085
:10420300546573742053696E7573206176656320FA
:104213005072696E742052616D20566964656F2017
:04422300200D0A0060
:10422700546573742061766563204269746D6170AB
:0E423700207061756C666A756A6F200D0A0052
:104245005465726D696E616C5F4E6F6B69615F3845
:0D4255007831365F31384632364B32320058
:104262006176656320466C6167204C69676E6531D3
:0A42720038636172733D310D0A00DC
:10427C0046696E2064652050726573656E74617456
:08428C00696F6E20200D0A008D
:104294000D0A20444542554720496D616765203920
:0742A400367836340D0A00E4
:1042AB00496E69742041444320706F7572204541FB
:0542BB0030200D0A0097
:1042C00054657374207175616472696C6C616765A3
:0542D00020200D0A0092
:1042D500ECF34A903595958F17C15C8BFDDBED8628
:0442E50072B33380FD
:1042E90020202020202020202020202020202020C5
:0442F9002020200061
:1042FD005175656C7175657320636572636C65735B
:04430D00200D0A0075
:024311000000AA
:0F431300E942004F4100B14100454200F3430031
:014322000F8B
:014323000099
:104324005465737420446961676F6E616C657320B2
:034334000D0A006F
:1043370050726573656E746174696F6E203A200DF3
:024347000A006A
:104349005465726D696E616C2052656164792020D3
:014359000063
:10435A0035656D206C69676E65202020202020203D
:01436A000052
:10436B0036656D206C69676E65202020202020202B
:01437B000041
:10437C0054657374205465726D696E65202120201C
:01438C000030
:10438D004541303D202020202020202020202020AD
:01439D00001F
:10439E0031323334353637383930313233343536CD
:0143AE00000E
:1043AF0034656D206C69676E6520202020202020E9
:0143BF0000FD
:1043C000496E64696365203A202020202020202047
:0143D00000EC
:1043D100313233343536373839303132333435369A
:0143E10000DB
:1043E20038656D206C69676E6520202020202020B2
:0143F20000CA
:1043F30031364632364B3232204C696238783136A8
:0144030000B8
:1044040056657273696F6E203A2031373038313116
:0144140000A7
:1044150037656D204C69676E65202020202020209F
:014425000096
:104426002B3401907F9D308BE7FF59850000007F7C
:10443600332072656374616E676C6573200D0A00C4
:0A444600496E64696365203D2000A3
:094450002020204541303D2000F0
:0844590052656164790D0A004F
:0844610052656164790D0A0047
:07446900313730383131001A
:05447000313030300086
:054475004F4B0D0A0091
:04447A0035303000A9
:04447E00373530009E
:020000040030CA
:0D00010028193CFFAE81FF0FC00FE00F403B
:0200000400F00A
:100000007061756C666A756A6F2E667265652E66BC
:10001000720D0A0000000000000000000000000057
:10002000496E6974204E6F6B6961204C43440D0A20
:1000300000000000000000000000000000000000C0
:1000400057726974652054657874206F6E204C4334
:1000500044200D0A00000000000000000000000025
:100060000000000000000000000000000000000090
:100070000000000000000000000000000000000080
:100080000000000000000000000000000000000070
:100090000000000000000000000000000000000060
:00000001FF
